
 Start         Length     Name                   Class
 0001:00000000 000019F4H .text                   CODE
 0002:00000000 0000003CH .data                   DATA
 0002:0000003C 0000004DH .bss                    BSS


Detailed map of segments

 0001:00000000 000000D6 C=CODE     S=.text    G=(none)   M=System   ACBP=A9
 0001:000000D8 000001EC C=CODE     S=.text    G=(none)   M=SysInit  ACBP=A9
 0001:000002C4 00000038 C=CODE     S=.text    G=(none)   M=Windows  ACBP=A9
 0001:000002FC 0000000E C=CODE     S=.text    G=(none)   M=Types    ACBP=A9
 0001:0000030C 00000038 C=CODE     S=.text    G=(none)   M=Messages ACBP=A9
 0001:00000344 0000000E C=CODE     S=.text    G=(none)   M=SysUtils ACBP=A9
 0001:00000354 0000000E C=CODE     S=.text    G=(none)   M=SysConst ACBP=A9
 0001:00000364 0000003E C=CODE     S=.text    G=(none)   M=Classes  ACBP=A9
 0001:000003A4 0000000E C=CODE     S=.text    G=(none)   M=ActiveX  ACBP=A9
 0001:000003B4 0000002E C=CODE     S=.text    G=(none)   M=TypInfo  ACBP=A9
 0001:000003E4 0000001E C=CODE     S=.text    G=(none)   M=Variants ACBP=A9
 0001:00000404 0000000E C=CODE     S=.text    G=(none)   M=VarUtils ACBP=A9
 0001:00000414 0000000E C=CODE     S=.text    G=(none)   M=RTLConsts ACBP=A9
 0001:00000424 0000000E C=CODE     S=.text    G=(none)   M=Graphics ACBP=A9
 0001:00000434 0000000E C=CODE     S=.text    G=(none)   M=Consts   ACBP=A9
 0001:00000444 000000F6 C=CODE     S=.text    G=(none)   M=Controls ACBP=A9
 0001:0000053C 0000000E C=CODE     S=.text    G=(none)   M=ActnList ACBP=A9
 0001:0000054C 0000000E C=CODE     S=.text    G=(none)   M=Contnrs  ACBP=A9
 0001:0000055C 0000000E C=CODE     S=.text    G=(none)   M=Math     ACBP=A9
 0001:0000056C 0000000E C=CODE     S=.text    G=(none)   M=ImgList  ACBP=A9
 0001:0000057C 00000038 C=CODE     S=.text    G=(none)   M=CommCtrl ACBP=A9
 0001:000005B4 0000012E C=CODE     S=.text    G=(none)   M=Forms    ACBP=A9
 0001:000006E4 0000000E C=CODE     S=.text    G=(none)   M=HelpIntfs ACBP=A9
 0001:000006F4 0000000E C=CODE     S=.text    G=(none)   M=MultiMon ACBP=A9
 0001:00000704 00000038 C=CODE     S=.text    G=(none)   M=Imm      ACBP=A9
 0001:0000073C 0000000E C=CODE     S=.text    G=(none)   M=Menus    ACBP=A9
 0001:0000074C 0000000E C=CODE     S=.text    G=(none)   M=Themes   ACBP=A9
 0001:0000075C 0000000E C=CODE     S=.text    G=(none)   M=UxTheme  ACBP=A9
 0001:0000076C 0000000E C=CODE     S=.text    G=(none)   M=SyncObjs ACBP=A9
 0001:0000077C 0000000E C=CODE     S=.text    G=(none)   M=ComCtrls ACBP=A9
 0001:0000078C 00000038 C=CODE     S=.text    G=(none)   M=ShlObj   ACBP=A9
 0001:000007C4 00000038 C=CODE     S=.text    G=(none)   M=UrlMon   ACBP=A9
 0001:000007FC 00000038 C=CODE     S=.text    G=(none)   M=WinInet  ACBP=A9
 0001:00000834 00000038 C=CODE     S=.text    G=(none)   M=RegStr   ACBP=A9
 0001:0000086C 00000038 C=CODE     S=.text    G=(none)   M=ShellAPI ACBP=A9
 0001:000008A4 0000000E C=CODE     S=.text    G=(none)   M=ListActns ACBP=A9
 0001:000008B4 0000000E C=CODE     S=.text    G=(none)   M=ExtCtrls ACBP=A9
 0001:000008C4 0000000E C=CODE     S=.text    G=(none)   M=StdCtrls ACBP=A9
 0001:000008D4 0000000E C=CODE     S=.text    G=(none)   M=WinHelpViewer ACBP=A9
 0001:000008E4 0000000E C=CODE     S=.text    G=(none)   M=StdActns ACBP=A9
 0001:000008F4 0000000E C=CODE     S=.text    G=(none)   M=Dialogs  ACBP=A9
 0001:00000904 0000000E C=CODE     S=.text    G=(none)   M=Printers ACBP=A9
 0001:00000914 00000038 C=CODE     S=.text    G=(none)   M=WinSpool ACBP=A9
 0001:0000094C 00000038 C=CODE     S=.text    G=(none)   M=CommDlg  ACBP=A9
 0001:00000984 00000038 C=CODE     S=.text    G=(none)   M=Dlgs     ACBP=A9
 0001:000009BC 0000000E C=CODE     S=.text    G=(none)   M=StrUtils ACBP=A9
 0001:000009CC 0000000E C=CODE     S=.text    G=(none)   M=Clipbrd  ACBP=A9
 0001:000009DC 0000000E C=CODE     S=.text    G=(none)   M=FlatSB   ACBP=A9
 0001:000009EC 0000000E C=CODE     S=.text    G=(none)   M=ToolWin  ACBP=A9
 0001:000009FC 00000038 C=CODE     S=.text    G=(none)   M=RichEdit ACBP=A9
 0001:00000A34 0000000E C=CODE     S=.text    G=(none)   M=ExtActns ACBP=A9
 0001:00000A44 0000000E C=CODE     S=.text    G=(none)   M=Registry ACBP=A9
 0001:00000A54 0000000E C=CODE     S=.text    G=(none)   M=IniFiles ACBP=A9
 0001:00000A64 0000000E C=CODE     S=.text    G=(none)   M=ExtDlgs  ACBP=A9
 0001:00000A74 0000000E C=CODE     S=.text    G=(none)   M=Buttons  ACBP=A9
 0001:00000A84 0000000E C=CODE     S=.text    G=(none)   M=Mapi     ACBP=A9
 0001:00000A94 0000000E C=CODE     S=.text    G=(none)   M=ComStrs  ACBP=A9
 0001:00000AA4 0000001E C=CODE     S=.text    G=(none)   M=DesignIntf ACBP=A9
 0001:00000AC4 0000000E C=CODE     S=.text    G=(none)   M=DesignMenus ACBP=A9
 0001:00000AD4 000000BE C=CODE     S=.text    G=(none)   M=DesignEditors ACBP=A9
 0001:00000B94 0000000E C=CODE     S=.text    G=(none)   M=Proxies  ACBP=A9
 0001:00000BA4 0000000E C=CODE     S=.text    G=(none)   M=DesignConst ACBP=A9
 0001:00000BB4 0000000E C=CODE     S=.text    G=(none)   M=ShellCtrls ACBP=A9
 0001:00000BC4 0000000E C=CODE     S=.text    G=(none)   M=ComObj   ACBP=A9
 0001:00000BD4 0000000E C=CODE     S=.text    G=(none)   M=ComConst ACBP=A9
 0001:00000BE4 0000000E C=CODE     S=.text    G=(none)   M=ShellConsts ACBP=A9
 0001:00000BF4 00000016 C=CODE     S=.text    G=(none)   M=FileCtrl ACBP=A9
 0001:00000C0C 000009D8 C=CODE     S=.text    G=(none)   M=RootEdit ACBP=A9
 0001:000015E4 000001B0 C=CODE     S=.text    G=(none)   M=ShellReg ACBP=A9
 0001:00001794 0000025D C=CODE     S=.text    G=(none)   M=dclshlctrls ACBP=A9
 0002:00000000 0000002C C=DATA     S=.data    G=DGROUP   M=SysInit  ACBP=A9
 0002:00001000 00000010 C=BSS      S=.bss     G=DGROUP   M=SysInit  ACBP=A9
 0002:00001010 00000004 C=BSS      S=.bss     G=DGROUP   M=Windows  ACBP=A9
 0002:00001014 00000004 C=BSS      S=.bss     G=DGROUP   M=Messages ACBP=A9
 0002:00001018 00000004 C=BSS      S=.bss     G=DGROUP   M=CommCtrl ACBP=A9
 0002:0000101C 00000004 C=BSS      S=.bss     G=DGROUP   M=Imm      ACBP=A9
 0002:00001020 00000004 C=BSS      S=.bss     G=DGROUP   M=ShlObj   ACBP=A9
 0002:00001024 00000004 C=BSS      S=.bss     G=DGROUP   M=UrlMon   ACBP=A9
 0002:00001028 00000004 C=BSS      S=.bss     G=DGROUP   M=WinInet  ACBP=A9
 0002:0000102C 00000004 C=BSS      S=.bss     G=DGROUP   M=RegStr   ACBP=A9
 0002:00001030 00000004 C=BSS      S=.bss     G=DGROUP   M=ShellAPI ACBP=A9
 0002:00001034 00000004 C=BSS      S=.bss     G=DGROUP   M=WinSpool ACBP=A9
 0002:00001038 00000004 C=BSS      S=.bss     G=DGROUP   M=CommDlg  ACBP=A9
 0002:0000103C 00000004 C=BSS      S=.bss     G=DGROUP   M=Dlgs     ACBP=A9
 0002:00001040 00000004 C=BSS      S=.bss     G=DGROUP   M=RichEdit ACBP=A9
 0002:00001044 00000004 C=BSS      S=.bss     G=DGROUP   M=RootEdit ACBP=A9
 0002:00001048 00000004 C=BSS      S=.bss     G=DGROUP   M=ShellReg ACBP=A9


  Address         Publics by Name

 0002:00001020       .1
 0002:00001024       .1
 0002:00001014       .1
 0002:00001028       .1
 0002:00001048       .1
 0002:00001008       .1
 0002:0000102C       .1
 0002:00001040       .1
 0002:0000103C       .1
 0002:00001018       .1
 0002:00001038       .1
 0002:0000101C       .1
 0002:00001030       .1
 0002:00001034       .3
 0002:00001010       .3
 0002:00001044       .4
 0001:000019CC       @GetPackageInfoTable
 0001:00000210       @InitPkg
 0001:00000274       @PackageLoad
 0001:000019D4       @PackageLoad
 0001:000019E0       @PackageUnload
 0001:00000280       @PackageUnload
 0001:00000110       AllocTlsBuffer
 0001:000005AC       CommCtrl
 0001:0000097C       CommDlg
 0001:000019EC       dclshlctrls
 0001:000009B4       Dlgs
 0001:0000149C       EditRoot
 0001:000001BC       ExitProcessTLS
 0001:00000194       ExitThreadTLS
 0001:000002C4       Finalization
 0001:00000984       Finalization
 0001:000015AC       Finalization
 0001:0000030C       Finalization
 0001:0000057C       Finalization
 0001:00000834       Finalization
 0001:00000704       Finalization
 0001:000009FC       Finalization
 0001:0000094C       Finalization
 0001:0000078C       Finalization
 0001:000007FC       Finalization
 0001:000007C4       Finalization
 0001:0000086C       Finalization
 0001:0000175C       Finalization
 0001:0000028C       Finalization
 0001:00000914       Finalization
 0001:000000D8       FreeLibrary
 0001:0000011C       GetTlsSize
 0002:00001004       HInstance
 0001:00000734       Imm
 0001:000001E0       InitializeModule
 0001:00000168       InitProcessTLS
 0001:00000124       InitThreadTLS
 0001:000000E0       LocalAlloc
 0001:000000E8       LocalFree
 0001:0000033C       Messages
 0002:00000004       Module
 0002:00001000       ModuleIsLib
 0002:00001001       ModuleIsPackage
 0001:00001044       PathIsCSIDL
 0001:000015E4       Register
 0001:00000864       RegStr
 0001:00000A2C       RichEdit
 0001:000015DC       RootEdit
 0001:00001098       RootPathEditor
 0001:0000089C       ShellAPI
 0001:0000178C       ShellReg
 0001:000007BC       ShlObj
 0001:000002BC       SysInit
 0001:000000F0       TlsAlloc
 0002:0000100C       tlsBuffer
 0001:000000F8       TlsFree
 0001:00000100       TlsGetValue
 0002:00000000       TlsIndex
 0002:FFBFD000       TlsLast
 0002:0000001C       TlsProc
 0001:00000108       TlsSetValue
 0001:00001574       TRootEditor.ExecuteVerb
 0001:0000158C       TRootEditor.GetVerb
 0001:000015A4       TRootEditor.GetVerbCount
 0001:000013F4       TRootPathEditDlg.btnBrowseClick
 0001:000013E8       TRootPathEditDlg.Button1Click
 0001:00001378       TRootPathEditDlg.Button2Click
 0001:00001374       TRootPathEditDlg.FormClose
 0001:00001294       TRootPathEditDlg.FormCreate
 0001:00001388       TRootPathEditDlg.rbUseFolderClick
 0001:000013B8       TRootPathEditDlg.rbUsePathClick
 0001:0000131C       TRootPathEditDlg.UpdateState
 0001:00001228       TRootProperty.Edit
 0001:00001288       TRootProperty.GetAttributes
 0001:000001EC       UninitializeModule
 0001:000007F4       UrlMon
 0001:000002F4       Windows
 0001:0000082C       WinInet
 0001:00000944       WinSpool


  Address         Publics by Value

 0002:FFBFD000       TlsLast
 0001:000000D8       FreeLibrary
 0001:000000E0       LocalAlloc
 0001:000000E8       LocalFree
 0001:000000F0       TlsAlloc
 0001:000000F8       TlsFree
 0001:00000100       TlsGetValue
 0001:00000108       TlsSetValue
 0001:00000110       AllocTlsBuffer
 0001:0000011C       GetTlsSize
 0001:00000124       InitThreadTLS
 0001:00000168       InitProcessTLS
 0001:00000194       ExitThreadTLS
 0001:000001BC       ExitProcessTLS
 0001:000001E0       InitializeModule
 0001:000001EC       UninitializeModule
 0001:00000210       @InitPkg
 0001:00000274       @PackageLoad
 0001:00000280       @PackageUnload
 0001:0000028C       Finalization
 0001:000002BC       SysInit
 0001:000002C4       Finalization
 0001:000002F4       Windows
 0001:0000030C       Finalization
 0001:0000033C       Messages
 0001:0000057C       Finalization
 0001:000005AC       CommCtrl
 0001:00000704       Finalization
 0001:00000734       Imm
 0001:0000078C       Finalization
 0001:000007BC       ShlObj
 0001:000007C4       Finalization
 0001:000007F4       UrlMon
 0001:000007FC       Finalization
 0001:0000082C       WinInet
 0001:00000834       Finalization
 0001:00000864       RegStr
 0001:0000086C       Finalization
 0001:0000089C       ShellAPI
 0001:00000914       Finalization
 0001:00000944       WinSpool
 0001:0000094C       Finalization
 0001:0000097C       CommDlg
 0001:00000984       Finalization
 0001:000009B4       Dlgs
 0001:000009FC       Finalization
 0001:00000A2C       RichEdit
 0001:00001044       PathIsCSIDL
 0001:00001098       RootPathEditor
 0001:00001228       TRootProperty.Edit
 0001:00001288       TRootProperty.GetAttributes
 0001:00001294       TRootPathEditDlg.FormCreate
 0001:0000131C       TRootPathEditDlg.UpdateState
 0001:00001374       TRootPathEditDlg.FormClose
 0001:00001378       TRootPathEditDlg.Button2Click
 0001:00001388       TRootPathEditDlg.rbUseFolderClick
 0001:000013B8       TRootPathEditDlg.rbUsePathClick
 0001:000013E8       TRootPathEditDlg.Button1Click
 0001:000013F4       TRootPathEditDlg.btnBrowseClick
 0001:0000149C       EditRoot
 0001:00001574       TRootEditor.ExecuteVerb
 0001:0000158C       TRootEditor.GetVerb
 0001:000015A4       TRootEditor.GetVerbCount
 0001:000015AC       Finalization
 0001:000015DC       RootEdit
 0001:000015E4       Register
 0001:0000175C       Finalization
 0001:0000178C       ShellReg
 0001:000019CC       @GetPackageInfoTable
 0001:000019D4       @PackageLoad
 0001:000019E0       @PackageUnload
 0001:000019EC       dclshlctrls
 0002:00000000       TlsIndex
 0002:00000004       Module
 0002:0000001C       TlsProc
 0002:00001000       ModuleIsLib
 0002:00001001       ModuleIsPackage
 0002:00001004       HInstance
 0002:00001008       .1
 0002:0000100C       tlsBuffer
 0002:00001010       .3
 0002:00001014       .1
 0002:00001018       .1
 0002:0000101C       .1
 0002:00001020       .1
 0002:00001024       .1
 0002:00001028       .1
 0002:0000102C       .1
 0002:00001030       .1
 0002:00001034       .3
 0002:00001038       .1
 0002:0000103C       .1
 0002:00001040       .1
 0002:00001044       .4
 0002:00001048       .1


Line numbers for dclshlctrls(dclshlctrls.dpk) segment .text

    41 0001:000019EC

Bound resource files

RootEdit.dfm
dclshlctrls.res
C:\DOCUME~1\~KOKOP~1\LOCALS~1\Temp\dtf295A.tmp


Program entry point at 0001:000019EC
